:1000000092C015C9ABC0AAC0A9C0A8C0A7C0A6C04D
:10001000A5C0B2CAA3C0A2C0A1C0A0C09FC09EC0BC
:100020009DC09CC09BC000000001010203030405A9
:100030000506070708090A0A0B0C0D0D0E0F101113
:10004000121213141516171818191A1B1C1D1E1F2F
:1000500020212122232425262728292A2B2C2D2E36
:100060002F303132333435363738393A3B3C3D3E28
:100070003F4041424345464748494A4B4C4D4E4F0D
:100080005051535455565758595A5B5D5E5F6061E5
:10009000626364666768696A6B6C6E6F70717273B5
:1000A00075767778797A7C7D7E7F8081838485867A
:1000B00087898A8B8C8D8F90919294959697989A38
:1000C0009B9C9D9FA0A1A2A4A5A6A7A9AAABACAEEC
:1000D000AFB0B1B3B4B5B6B8B9BABBBDBEBFC1C29B
:1000E000C3C4C6C7C8CACBCCCDCFD0D1D3D4D5D743
:1000F000D8D9DADCDDDEE0E1E2E4E5E6E8E9EAECE5
:10010000EDEEF0F1F2F4F5F6F8F9FAFCFDFEFFFF82
:10011000FFFFFFFFFFFFFFFFFFFFFFFFFFFFFFFFEF
:10012000FFFFFFFFFFFF11241FBECFE5D4E0DEBFBE
:10013000CDBF11E0A0E6B0E0E4E1F8E102C0059037
:100140000D92A837B107D9F713E0A8E7B1E001C0D5
:100150001D92A634B107E1F7B8D45ACB51CF482F3E
:1001600090E820E030E0FB01E20FF31F892F8423A9
:10017000808396952F5F3F4F28303105A1F7089572
:10018000262F2058332727FD3095992787FD9095F6
:10019000281B390B442737FD4095542FCA01B9015C
:1001A00028E139E740E050E09DDA20E03DE740E01B
:1001B00050E0B7DA8FEF223838071CF421E83FEF20
:1001C00005C02038310514F02FE730E0C90108954B
:1001D0002F923F924F925F926F927F928F929F9257
:1001E000AF92BF92CF92DF92EF92FF920F931F9345
:1001F000DF93CF93CDB7DEB72A970FB6F894DEBF63
:100200000FBECDBF6C017A876987FC018681807142
:10021000FB018183F60186818870E985FA858583F3
:10022000F60186818078E985FA858187F6018681E5
:100230008170E985FA858587F60186818072E98576
:10024000FA85818BF60186818074E985FA85858B34
:100250007896F887EF83F60183818058EF81F885DF
:100260008183F60183818058E985FA85858FB09670
:10027000FE83ED83F60182818058ED81FE818183CA
:10028000F60182818058E985FA8585A3F601878188
:100290008170E985FA8581A7F60187818270E985F9
:1002A000FA8585A7F60187818870E985FA8581AB93
:1002B000F60187818470E985FA8585ABF896FC8321
:1002C000EB8389859A85CC969A838983809178017E
:1002D000F601608155DF1C014C01AA2497FCA09413
:1002E000BA2C80917901F60161814ADF2C016624E4
:1002F00057FC6094762C97FF03C0909581959F4F93
:10030000682F70E080E090E0A5019401EBD920E82F
:100310003EE340E050E005DA79018A01E80CF91C7F
:100320000A1D1B1DC10137FE03C0909581959F4F8B
:10033000682F70E080E090E0A3019201D3D920E81B
:100340003EE340E050E0EDD9240D351D461D571D1C
:10035000F2E8EF16FFEFFF06FFEF0F07FFEF1F07B3
:100360004CF491E8E92E9FEFF92E9FEF092F9FEFB4
:10037000192F0BC080E8E816F104010511052CF0D7
:100380008FE7E82EF12C012D112D22389FEF390730
:100390009FEF49079FEF59072CF421E83FEF4FEFFC
:1003A0005FEF09C0203831054105510524F02FE7E2
:1003B00030E040E050E0EB81FC81E182E981FA81AC
:1003C000218389859A85805C9F4F9A878987F6016A
:1003D00086818470E985FA8581833496FA87E98776
:1003E000F60186818270E985FA8581833496FA87E1
:1003F000E987E981FA818181E985FA8581833496EB
:10040000FA87E987E981FA818181E985FA85818323
:100410003496FA87E987EB81FC818181E985FA8549
:1004200081833496FA87E987EB81FC818181E985B4
:10043000FA8581833496FA87E987F60184818058AA
:10044000E985FA8581833496FA87E987F601858103
:100450008058E985FA8581833496FA87E987ED81AA
:10046000FE818181E985FA8581833496FA87E9875F
:10047000EF81F8858181E985FA8581832A960FB617
:10048000F894DEBF0FBECDBFCF91DF911F910F91CA
:10049000FF90EF90DF90CF90BF90AF909F908F90A4
:1004A0007F906F905F904F903F902F900895CF93E3
:1004B000DF93C0E0DAEFCE010197F1F7E091FC01A4
:1004C000F091FD010484F585E02D0995E091FC0192
:1004D000F091FD010684F785E02D0995882359F3F5
:1004E000E091FC01F091FD010088F189E02D8EEF93
:1004F00091E009958EEF91E06EEA70E069DE20E010
:1005000030E08091AF00882311F021E030E080914D
:10051000B300811122608091EF00811124608091ED
:10052000F300811128608091B700811120618091D2
:10053000BF00811120628091C300811120648091ED
:10054000D700811120688091DB008111316080919A
:10055000DF00811132608091E3008111346080916D
:10056000BB0081113860E0917C01F0917D01E227B0
:10057000F32741E050E060E070E0CA018E239F2342
:10058000892B69F0CA0182239323892B41F0309390
:100590007D0120937C01CA01DF91CF910895440F22
:1005A000551F6F5F7F4F6C30710539F730937D01B8
:1005B00020937C0180CFDF92EF92FF920F931F93E5
:1005C000CF93DF937B01D42E052F8032910519F054
:1005D000EB0110E80EC0FB0180819181FFEF8F3F9E
:1005E0009F0709F451C00196FB019183808349C0A4
:1005F0005EDF88309105D1F1893091054CF482306D
:10060000910561F18430910569F1019789F723C063
:100610008032910579F1F8E080309F07A9F1409789
:1006200039F7103841F0188319828D2D902F9C01D5
:10063000E90110E8DDCFF70180819181FFEF8F3F65
:100640009F0711F10196F701918380838D2D902FE3
:100650009C01E901CDCF110F110FCACF110F110F5E
:100660001F5FC6CF110F110F1E5FC2CF110F110FE9
:100670001D5FBECFCE15DF0539F0103811F018839D
:10068000198220E030E002C02FEF3FEFC901DF9177
:10069000CF911F910F91FF90EF90DF900895CF932E
:1006A000DF93DC01EB0120E011969C9111971396EA
:1006B0008C911397981321E02883FD01349620E054
:1006C00091818381981321E02983FD01389620E0F0
:1006D00091818381981321E02A83FD013C9620E0DB
:1006E00091818381981321E02B83FD01B89620E04E
:1006F00091818381981321E02C83FD01BC9620E039
:1007000091818381981321E02D83FD01F09620E0F3
:1007100091818381981321E02E83FD01F49620E0DE
:1007200091818381981321E02F8318861986FD011A
:10073000709620E091818381981321E02A87FD0142
:10074000749620E091818381981321E02B87FD012D
:10075000789620E091818381981321E02C87FD0118
:100760007C9620E091818381981321E02D87FD0103
:10077000B09620E091818381981321E02E87FD01BE
:10078000B49620E091818381981321E02F87D99638
:100790003C91D997DD962C91DD97FD01E05CFF4FF0
:1007A00091818381981709F4922FFD01EC5BFF4F33
:1007B00051818381581709F4592FFD01E85BFF4FE0
:1007C00091818381981709F4932FFD01E45BFF4F1A
:1007D00041818381481709F4492FFE01709690E802
:1007E0009E01285E3F4F892F842381939695E217BF
:1007F000F307C9F7252F209590E8BE01605E7F4F73
:10080000892F822381939695E617F707C9F7DF9121
:10081000CF910895A6E0B2E0E0E6F0E028E3019091
:100820000D922150E1F79C012150304024303105D8
:10083000C0F488E390E0289FF001299FF00D389FD5
:10084000F00D1124EA5BFD4F80818F3F19F42FEFEB
:100850003FEF09C0A6E0B2E088E301900D9281501D
:10086000E1F720E030E0C90108959C0121503040BB
:100870002430310598F488E390E0289FF001299F07
:10088000F00D389FF00D1124EA5BFD4FA6E0B2E0B9
:1008900088E30D9001928150E1F79CD6089581E0A4
:1008A00090E048D604DE22E080309207D9F022E0C2
:1008B000813092073CF48038910571F0805091406E
:1008C00041F40DC024E08030920779F080509840C8
:1008D00081F02FEF3FEF12C081E090E008C082E08E
:1008E00090E005C083E090E002C084E090E0BDDFCE
:1008F00003C080E090E08EDF20E030E0C901089581
:10090000DF92EF92FF920F931F93DF93CF9300D06C
:1009100000D0CDB7DEB78FEF9FEF9A8389839C839A
:100920008B83DFB6F894F7D585E090E003D600E03E
:100930001AEFE091FC01F091FD010484F585E02DB2
:100940000995E091FC01F091FD010088F189E02D0D
:100950008EEF91E009958EEF91E06EEA70E038DC61
:100960008091BB00882321F0C8010197F1F7E1CF06
:10097000B3E0EB2EF12CEC0EFD1E8E010F5F1F4F2E
:1009800096DD9C018032910509F443C081329105C6
:1009900094F48430910509F43CC08530910524F429
:1009A0000197029768F735C08830910591F1803141
:1009B000910531F72EC081E020303807D9F081E071
:1009C000213038073CF420343105F1F0203831056E
:1009D000B9F60DC084E02030380791F088E020306F
:1009E000380709F443C02050324051F606C081E078
:1009F00090E008C082E090E005C083E090E002C093
:100A000084E090E007DF01C04ADF8F5F9F4F71F500
:100A10001AC0C901B801A701CEDD8F5F9F4F99F0C1
:100A200069817A818FEF6F3F780769F04B815C8134
:100A30002FEF4F3F520739F086E092E0D6D481E0A5
:100A400090E078D59DCF83E090E074D581E090E090
:100A500065D588E59BE120E931E0F9013197F1F7AF
:100A60000197D9F780E090E059D503C083E090E08A
:100A700061D5E8D5DFBE0F900F900F900F90CF910A
:100A8000DF911F910F91FF90EF90DF900895FC018F
:100A90008585882391F094D5882399F080917A01F7
:100AA00090917B01019690937B0180937A01069748
:100AB00044F026DF21E030E006C010927B01109266
:100AC0007A0120E030E0C9010895CCD09093FD0177
:100AD0008093FC0111BA82B38B6F82BB889A14BADF
:100AE0008FEF85BB85B7886085BF85B78B7F85BF56
:100AF0008BB780648BBF20EB31E0C90160E070E010
:100B000040E250E058D620ED31E0C90160E070E0ED
:100B100040E250E050D695E09093F0011092F10140
:100B200082E08093F2019093F3011092F40110920D
:100B3000F5017894F0D456D5892B19F082E090E035
:100B4000F9D48091450290E065DE31D5E091FC0159
:100B5000F091FD010284F385E02D0995909A88E8D3
:100B600093E120E931E0F9013197F1F70197D9F7E5
:100B7000E091FC01F091FD010484F585E02D0995DB
:100B8000E091FC01F091FD010088F189E02D8EEFEC
:100B900091E009958091FE018058809378018091C1
:100BA000FF018058809379018EEF91E06EEA70E04A
:100BB0000FDB8091BB00882319F08EEA90E0A0DE65
:100BC000909840D58091F601882319F01092F60193
:100BD00047D575D58823B1F3909AE1D4E091FC0113
:100BE000F091FD010484F585E02D0995DCD4909801
:100BF000E091FC01F091FD010684F785E02D099557
:100C0000882361F1909AE091FC01F091FD01008848
:100C1000F189E02D8EEF91E009958EEF91E06EEA7B
:100C200070E0D6DA86E092E06EEA70E04AE151E0E8
:100C300013D48091F701882319F460ED71E002C0AC
:100C400060EB71E08AE191E02ADD8091F70190E0AC
:100C5000882309F491E09093F70190988EEA90E050
:100C600016DFB0CF88E990E00895009741F0DC01ED
:100C7000EEE7F1E088E001900D928150E1F7A6E8FF
:100C8000B1E0EEE7F1E088E001900D928150E1F7EC
:100C900008958091AC009091AD00892B31F01092B5
:100CA000AD001092AC0081E008958EE791E066E817
:100CB00071E048E050E072D508950F931F93DF93E1
:100CC000CF93CDB7DEB7C850D1400FB6F894DEBF92
:100CD0000FBECDBF80E013D288EC90E00197F1F712
:100CE000FE01399680E0EF93FF9300E810E41023B3
:100CF000C9F00000A39A00000000000000000000FE
:100D000000000000000000000000000000000000E3
:100D10000000A3983CE03A95F1F70000000006952A
:100D200081F0E4CFA39A3FE03A95F1F70000A39851
:100D3000000000000000000000000000069509F01F
:100D4000D5CFA39800E813E01023C9F00000A39AC0
:100D50000000000000000000000000000000000093
:100D6000000000000000000000000000A3983CE02C
:100D70003A95F1F700000000069581F0E4CFA39AC0
:100D80003FE03A95F1F70000A39800000000000052
:100D9000000000000000069509F0D5CFA39800E8F8
:100DA000182F1023C9F00000A39A000000000000D3
:100DB0000000000000000000000000000000000033
:100DC000000000000000A3983CE03A95F1F7000015
:100DD0000000069581F0E4CFA39A3FE03A95F1F741
:100DE0000000A398000000000000000000000000C8
:100DF000069509F0D5CFA398000000000000000080
:100E0000A39A0000000000000000000000000000A5
:100E100000000000000000000000000000000000D2
:100E20000000A39800000000000000000000000087
:100E30000000000013B31870E9F330E40FE30A95E3
:100E400019F013B31870D9F788278095FF91EF91A7
:100E5000C198EF93FF93882700270395B1F09B99E2
:100E6000FCCF000008C00027039579F09B99FCCFC8
:100E7000839551F001930027039539F09B9BFCCF9C
:100E8000839511F00193EFCF0000FF91EF9181382E
:100E900021F081E080938E0112C1DF01AE0147573E
:100EA0005F4F20E090818181981708F421E02D9315
:100EB0003296E417F507A9F7FE01319688E0DF01C5
:100EC0001D928A95E9F74981FE01799620E030E08C
:100ED00060E870E08081882339F0CB01022E02C0E7
:100EE000959587950A94E2F7482B2F5F3F4F3196EF
:100EF0002830310579F749834A81FE01B19620E017
:100F000030E060E870E08081882339F0CB01022E68
:100F100002C0959587950A94E2F7482B2F5F3F4FC3
:100F200031962830310579F740954A834B81FE018F
:100F3000B99620E030E060E870E08081882339F0E5
:100F4000CB01022E02C0959587950A94E2F7482BB3
:100F50002F5F3F4F31962830310579F74B834C8115
:100F6000FE01F19620E030E060E870E080818823A7
:100F700011F080E007C0CB01022E02C09595879545
:100F80000A94E2F7482B2F5F3F4F31962830310506
:100F900069F74C834D81FE01F99620E030E060E86E
:100FA00070E08081882339F0CB01022E02C0959534
:100FB00087950A94E2F7482B2F5F3F4F31962830F0
:100FC000310579F740954D834E81FE01EF5BFF4F70
:100FD00020E030E060E870E08081882339F0CB01C8
:100FE000022E02C0959587950A94E2F7482B2F5F51
:100FF0003F4F31962830310579F740954E834F8128
:10100000FE013C9620E030E061E070E080818823C2
:1010100039F0CB01022E02C0880F991F0A94E2F723
:10102000482B2F5F3F4F31962530310579F7FE0170
:10103000729620E030E060E270E08081882339F031
:10104000CB01022E02C0880F991F0A94E2F7482BA9
:101050002F5F3F4F31962330310579F74F83488515
:10106000FE01759620E030E061E070E08081882329
:1010700039F0CB01022E02C0880F991F0A94E2F7C3
:10108000482B2F5F3F4F31962430310579F7898106
:1010900080937E018A8180937F018B818093800180
:1010A0008C81809381018D81809382018E818093D8
:1010B00083018F81809384014093850180E0C85F24
:1010C000DE4F0FB6F894DEBF0FBECDBFCF91DF91DC
:1010D0001F910F91089510928E01EFDD90E08091A5
:1010E0008E01882309F491E0892F08958FB7F89431
:1010F000B99AC198A398AB988FBFDFDD08950F937D
:101100001F93DF93CF93CDB7DEB7C154D0400FB656
:10111000F894DEBF0FBECDBFFE013196EF93FF9373
:1011200000E8182F1023C9F00000A39A0000000067
:1011300000000000000000000000000000000000AF
:101140000000000000000000A3983CE03A95F1F791
:1011500000000000069581F0E4CFA39A3FE03A95A5
:10116000F1F70000A398000000000000000000005C
:101170000000069509F0D5CFA398000000000000FC
:1011800000000000000000000000A39A0000000022
:10119000000000000000000000000000000000004F
:1011A0000000000000000000A39830E20FEF0A9555
:1011B00029F113B31072D9F7C198000000000000A4
:1011C000000000000000000000000000000000001F
:1011D000000000000000000023B3C19A2870219392
:1011E0003A9539F00FEF0A9549F023B32870F1F6DC
:1011F000FACF882705C0C19A832F02C0882780951F
:10120000FF91EF91C1988F3F19F020E030E002C0CC
:101210002FEF3FEFC901CF5BDF4F0FB6F894DEBF72
:101220000FBECDBFCF91DF911F910F9108951F92F7
:101230001FB6EF93FF934F930F931F937F93EFE8A6
:10124000F1E001E20EC015E11A95D9F040B3447007
:10125000D9F70000000000000000000000000000BE
:10126000000034D0000040B30000447041930A9560
:1012700039F015E11A9529F040B34470D9F3E3CF62
:1012800004C041E2401B493049F07F911F910F910A
:101290004F91FF91EF911FBE1F90189541E0E6EF2F
:1012A000F1E04083EFE8F1E015D0442359F04130FC
:1012B00059F04F3F29F0909A000000009098E5CF38
:1012C00034D0E3CF1FD0E1CF43D0DFCF12E01A9567
:1012D000F1F708950F931F93442700E8119111230C
:1012E00009F0402B0695D1F71F910F9108950F93A8
:1012F0001F9300E8142F102311930695D9F71F911F
:101300000F910895AF93BF93A0EFB1E0EFE8F1E044
:101310004D91EDDF4D91EBDF4D91E9DFBF91AF9145
:10132000EFE8F1E078E121D00895AF93BF93A3EF08
:10133000B1E0EFE8F1E04D91DADF4D91D8DF4D916A
:10134000D6DFBF91AF91EFE8F1E078E10ED00895DC
:10135000E7EFF1E07081772319F4E0EBF1E002C0F0
:10136000E0EDF1E070E201D008953F934F937F9359
:1013700031913323E1F400008A9A4FE04A95F1F766
:1013800000008A9842E04A95F1F77A9589F70000C3
:10139000000000000000000000008A9A44E04A9526
:1013A000F1F700008A987F914F913F9108958A9AB2
:1013B00044E04A95F1F7000000008A984CE04A9515
:1013C000F1F7000000007A9599F600000000000097
:1013D0000000000000008A9A44E04A95F1F70000FE
:1013E0008A987F914F913F910895FC0109C09927F8
:1013F00087FD90958617970711F4418308953296DB
:1014000080818F3FA1F70895FC018081823011F027
:1014100080E0089581810895FC018081833041F04E
:10142000843091F0813011F020E014C0218112C08D
:101430003281818137FF04C020E038175CF009C099
:1014400020E083173CF005C020E09181828189175C
:101450000CF021E0822F0895CF92DF92EF92FF925D
:101460000F931F93CF93DF938C017B016A01FA01E5
:1014700003C083818183349680818823D1F73DC066
:10148000282F332727FD3095F8018181C82FDD27CC
:10149000C7FDD095CC0FDD1FCC0FDD1FCC0DDD1DA2
:1014A0008881823081F08330D1F0813021F5220FA4
:1014B000331F220F331FC701820F931FADDF9981A6
:1014C000982B998318C0F901EE0FFF1FEE0FFF1F35
:1014D000EE0DFF1D8081823071F481810BC0220FDF
:1014E000331F220F331FC701820F931F95DF8823FD
:1014F00011F08A8189830E5F1F4FF80180818F3F31
:1015000009F0BECFDF91CF911F910F91FF90EF9027
:10151000DF90CF900895C198B99A0895892B11F45E
:101520001FBC089581E88FBD8AE08EBD1BBC8FE192
:101530008ABD08950F931F93CF93DF93EC0100E9C9
:1015400011E081E090E0EADF80EB94E0F801319770
:10155000F1F70197D9F780E090E0E0DF84EF91E0C8
:10156000F8013197F1F70197D9F7219751F7DF91FA
:10157000CF911F910F9108951F920F920FB60F9266
:1015800011248F938091F8018C3318F48F5F80932E
:10159000F8018F910F900FBE0F901F90189589B78B
:1015A0008E7F89BF089589B7816089BF089585E0DE
:1015B00083BF12BE89B7816089BF1092F801089578
:1015C0008091F8018C3310F480E008951092F801B6
:1015D00081E008958EE392E060E070E048E051E041
:1015E00001D108958EE392E060E070E048E051E0C0
:1015F000E9D08EE392E06EE671E047E050E0CED0B5
:10160000009719F420E030E01BC0AEE3B2E0EEE654
:10161000F1E087E001900D928150E1F710924502D0
:1016200086E492E06FEF70E040E051E0C4D08EE3DA
:1016300092E060E070E048E051E0D4D021E030E09A
:10164000C90108951FBC83E08EBD1DBC1CBC109257
:10165000FB0186ED96E09093FA018093F9010895DD
:1016600008B602FE04C088B7846088BF1AC08CB573
:101670009DB524E0833E9207D0F027E0813D92079C
:1016800018F08E5E924002C086ED96E09093FA01CB
:101690008093F9018091F9019091FA01825E944062
:1016A00030F486ED96E09093FA018093F9011DBC29
:1016B0001CBC88B7846088BF1092FB01089580919C
:1016C000FB01882369F42CB53DB58091F901909117
:1016D000FA012817390720F081E08093FB01089573
:1016E00080E00895629FD001739FF001829FE00D1A
:1016F000F11D649FE00DF11D929FF00D839FF00D91
:10170000749FF00D659FF00D9927729FB00DE11D3C
:10171000F91F639FB00DE11DF91FBD01CF01112419
:10172000089597FB092E05260ED057FD04D014D03E
:101730000AD0001C38F450954095309521953F4FC4
:101740004F4F5F4F0895F6F790958095709561958E
:101750007F4F8F4F9F4F0895A1E21A2EAA1BBB1BEC
:10176000FD010DC0AA1FBB1FEE1FFF1FA217B3076D
:10177000E407F50720F0A21BB30BE40BF50B661F83
:10178000771F881F991F1A9469F760957095809547
:1017900090959B01AC01BD01CF010895FB01DC01D7
:1017A00004C08D910190801921F441505040C8F738
:1017B000881B990B0895DC0101C06D934150504086
:1017C000E0F70895DC01CB01FC01E199FECF06C0F2
:1017D000FFBBEEBBE09A31960DB20D9241505040E6
:1017E000B8F70895DC01CB0102C02D9105D041501E
:1017F0005040D8F70895262FE199FECF9FBB8EBBAE
:101800002DBB0FB6F894E29AE19A0FBE01960895A7
:04181000F894FFCF7A
:10181400000001010202030304040505060607078C
:10182400080809090A0A0B0B0C0C0D0D0E0E0F0FFC
:101834001014111412141314141415141604170587
:10184400181419141A14FFFF080000000000000007
:10185400000076085D06490635066B0801000100A4
:101864000000010000000100000001000000010070
:101874000000010000000300E0000300200003005A
:10188400E00003002000010000000100000001004E
:10189400000001000000020000000200000001003E
:1018A400000001000000030020000300E00003002A
:1018B40020000300E00004002000040020000200D7
:1018C4000000020000000000000001000000010010
:1018D4000000010000000100000001000000010000
:1018E40000000100000001000000010000000100F0
:1018F40000000100000001000000010000000100E0
:101904000000020000000200000003008100030048
:101914007F000300810003007F00000000004743B4
:08192400324E3634763100002A
:00000001FF
